:1000000010308A0000280000D3346D38EC32202AEA
:10001000E832F236EF36653AE8327210A0060A008E
:10002000533A613B3A10A53A64147039EF316537A1
:10003000F430A9060A00533A613B3A10A53A641419
:100040007039EF316537F430A9060A00533A613B45
:100050003A10A53A64147039EF316537F430A906C7
:100060000A00533A613B3A10A53A64147039EF31F3
:100070006537F430A9060A00533A613B3A10A53AB5
:1000800064147039EF316537F430A9060A00533A29
:10009000613B3A10A53A64147039EF316537F4309A
:1000A000A9060A00533A613B3A10253220147039F0
:1000B000EF316537F430A9060A00533A613B781DE9
:1000C000A0124C322838F237E3326E3AE1140D05B3
:1000D0000000533A613B791DA0124C322838F237A8
:1000E000E3326E3AE1140D050001533A613B7A1D8B
:1000F000A0124C322838F237E3326E3AE1140D0583
:100100000001F9177A10A51830173233A0060A003B
:10011000613A6137A01231182E1966100D050001E1
:1001200075346536A01231182E1966100D050000C1
:10013000A013200883168700831287130830F80065
:10014000A1280000F817B228F813C90C0318871764
:10015000031C87137817B2287813F80BA528B0284A
:10016000000087173F308400840BB4280000F81B80
:10017000A428781BAC280800831603178C170C14CE
:100180000000000083120C087F39031900290313B3
:10019000BC0003170D080313BD0003170F0803135A
:1001A000BE003C08C90098203D0803178D000313CA
:1001B0003E0803178F0083168C170C1400000000F4
:1001C00083120C0D0E0D7F39031900290313BC0097
:1001D00003170D080313BD0003170F080313BE0018
:1001E0003C08C90098203D0803178D0003133E0802
:1001F00003178F008D0A03198F0A0313BC280317F6
:1002000003138A110A166D280830F80000008711C0
:10021000A01120088316870000008312BC0D07126E
:10022000031C182920162008831687001C29831216
:10023000201220088316870000008312A0152008D2
:10024000831687008312871D2329F80B06290000D7
:100250008711A01120088316870000008312201642
:10026000200883168700000000008312A0152008D4
:10027000831687008312871D3B29F8010000071AA7
:1002800078148711A01120088316870083120712A3
:100290002012200883168700831208000830BD0052
:1002A0007708BE00201620088316870000008312FE
:1002B000A0152008831687008312871D5D29071A61
:1002C0000314071E0310F80D0000A0112008831668
:1002D000870083128711BD0B522920162008831630
:1002E00087000000831207123E0803197C292012A0
:1002F00020088316870083120000A01520088316AB
:1003000087008312871D822900008711A011200811
:10031000831687000000831207122012200883161C
:10032000870083120800831603178C170C14000033
:1003300000000318C22983120C087F390313BE0082
:1003400003170D080313BF0003170F080313C000A2
:100350003E08C90098203F0803178D00031340088A
:1003600003178F0083168C170C14000000008312F3
:100370000313BD0BBC29BF2983160317C229E1292A
:100380008316031783120C0D0E0D7F390313BE0065
:1003900003170D080313BF0003170F080313C00052
:1003A0003E08C90098203F0803178D00031340083A
:1003B00003178F008D0A03198F0A03100313BD0B57
:1003C000932908004408F80143020318EA29430866
:1003D000F700F629F7010830C500C30DF70D4408F2
:1003E00077020318F700F80DC50BED29080078080F
:1003F0003C08C3006430C400E2217708BC007808E0
:100400003030031D0A2ABD1C112ABD19112A3D1ABC
:1004100020300D2ABD113D123D14F8077808C9009F
:1004200098203C08C3000A30C400E2217708BC00D1
:1004300078083030031D222ABD19262A3D1C262AA1
:100440003D1A2030F8077808C90098203030BC07E2
:100450003C08C900982008003D083F068039C100CB
:10046000BD1F372ABC09BD09BC0A0319BD0ABF1F3D
:100470003E2ABE09BF09BE0A0319BF0AF801F901E5
:10048000F701FA013F08031D482A3E080319622AB2
:100490001030C0000310BC0DBD0DF70DFA0D3F0864
:1004A0007A02031D552A3E087702031C5E2A3E0885
:1004B000F702031CFA033F08FA020314F80DF90DC2
:1004C000C00B4A2AC11F692AF809F909F80A031959
:1004D000F90A080020303E1E3030BF003D08F7000A
:1004E000BD1F792AF709F70A7708BD002D30BF0034
:1004F000BE173D08C3006430C400E2217708BD0088
:1005000030307807C0003D08C3000A30C400E22143
:1005100030307707C20030307807C1003F08F7005D
:10052000BE1D942ABE1F3E113E1AA12ABE1FBC2A20
:100530003E19BC2A7708C000BE18BC2A7708C10043
:10054000BC2A30304002031DBC2A7708C00020308E
:10055000BF00BE1DAF2A3E11BE14BE1FBE103030FC
:100560004102031DBC2A7708C1002030C000BE1D17
:10057000AF2ABE10BE1F3E103E1DC12A3F08C90053
:100580009820BE1CC62A4008C90098203E1CCB2AD1
:100590004108C90098204208C90098208A110A160B
:1005A000B62CC4010408C3004410831B4414BD1FAF
:1005B000E12AC317431EC30ABC09BD09BC0A0319BB
:1005C000BD0A3D0EF038BF00BF07E23EC000323E1C
:1005D000C2003D080F39C007C007C207E93EC1008D
:1005E000C107C1073C0E0F39C107C207C10DC20DBB
:1005F000C209C20D3C080F39C207BF0D0730BE004B
:100600000A30C207C103031C012BC107C003031C2E
:10061000052BC007BF03031C092BBF07BE03031C28
:100620000D2B3E30840083130730430543138403AE
:100630004305031D222B431A840A431A222B203020
:10064000F7003F2B840742300402031943170008C8
:10065000F700031D332B431B332B431A4D2BC319B8
:10066000332B20303E2BC31F3B2B2D30F700840350
:100670004313C3133F2BC31543123030F707BD019B
:100680000408BC003D10831B3D147708C900982066
:100690003C08840083133D188317840A431F232BCF
:1006A00008008E30F7004108F8004008F900FA0110
:1006B000C11F5F2BF809F909F90A0319F80AF808AC
:1006C000031D6C2B7908F800F9010830F702F808CF
:1006D000031D6C2BF701752B0310F81B732BF90D01
:1006E000F80DF7036C2BC11FF8130800510803190C
:1006F0003B2CDD00550803193B2CDD02031C852B28
:100700007F30DD0703183B2C8B2B8130DD02031C6F
:100710003B2C03193B2C5D08F700F801F901FA01A5
:10072000DC015208DB00DB175308DA005408D9005B
:100730001930DD005808D9020318AE2B0130DA0257
:100740000318AE2BDB020318AE2BDC020318AE2B12
:10075000DC0ADB0ADA0A5808D907E02B5708DA0264
:100760000318C92B0130DB020318C92BDC02031864
:10077000C92BDC0ADB0A5708DA075808D907031C1B
:10078000E02BDA0A031DE02BDB0A031DE02BDC0A59
:10079000E02B56088038DB020318DF2B0130DC0227
:1007A0000318DF2BDC0A56088038DB075708DA0706
:1007B000031CBD2BDB0A031DBD2BDC0ABD2B7A14E9
:1007C000DD0BE32BEE2B0310D90DDA0DDB0DDC0D69
:1007D0000310FA0DF90DF80DDE0D9A2B5E1CF62BA9
:1007E0000310F80CF90CFA0CDE0CF92BF7030319C3
:1007F0003B2CDE1B222C0310D90DDA0DDB0DDC0D9A
:100800005808D90203180E2C0130DA0203180E2CF6
:10081000DB0203180E2CDC02031C312C5708DA0211
:100820000318192C0130DB020318192CDC02031CFD
:10083000312C56088038DB020318222C0130DC02F0
:10084000031C312CFA0A031D312CF90A031D312C2B
:10085000F80A031D312CF70A03193B2CF80CF90C8C
:10086000FA0C5208DD005608DD06DD1F392CF8179A
:100870003F2CF8133F2CF701F801F901FA010800A9
:1008800051080319B02CD90055080319B02CD90709
:100890000318512C7F30D902031CB02C0319B02C43
:1008A000552C8130D9070318B02C5908F700F801EE
:1008B000F901FA015208DD00DD175308DC00540885
:1008C000DB001830D900DA015B1C7E2C5808FA07CF
:1008D000031C702CF90A031D702CF80A0319DA178F
:1008E0005708F907031C772CF80A0319DA1756087A
:1008F000D300D3175308F8070318DA17DA0DF80CEA
:10090000F90CFA0CDD0CDC0CDB0C0310D90B632C9E
:100910000130F7070318B02CF81B952CDD0DFA0DEC
:10092000F90DF80DF7030319B02CDD1FA62CFA0AF8
:10093000031DA62CF90A031DA62CF80A031DA62CDC
:10094000F80CF90CFA0CF70A0319B02C5208DA006B
:100950005608DA06DA1FAE2CF817B42CF813B42CAC
:10096000F701F801F901FA010800F701F801F901AE
:10097000FA01D101D201D301D40150084F044E0431
:100980004D040319F32C2030D5000310C90DCA0DF6
:10099000CB0DCC0DD10DD20DD30DD40D500854027A
:1009A000031DDC2C4F085302031DDC2C4E085202A1
:1009B000031DDC2C4D085102031CED2C4D08D10207
:1009C0004E08031C4E0FD2024F08031C4F0FD302D8
:1009D0005008031C500FD4020314F70DF80DF90D45
:1009E000FA0DD50BC52C5130840083130800040880
:1009F000C1004008C3000319162D3F08D4003E086B
:100A0000D3003D08D2003C08D100D801D7012030E6
:100A1000D6008230D50040247A08BF007908BE0095
:100A20007808BD007708BC00C30BFD2C3F08CC0044
:100A30003E08CB003D08CA003C08C9004908B63C46
:100A4000C900FA014A08CD00CA170310CA0CCB0C22
:100A5000CC0CFA0CF90CF80CF70CC90B252DCD1F9A
:100A60003C2DF709F809F909FA09F70A0319F80AF8
:100A70000319F90A0319FA0A7A08BF007908BE00B7
:100A80007808BD007708BC00BF1F532DC103C116F5
:100A9000BC09BD09BE09BF09BC0A0319BD0A031977
:100AA000BE0A0319BF0A3B30C8009A30C700CA30DB
:100AB000C600C5010A30C30040080319C10A3F0837
:100AC000CC003E08CB003D08CA003C08C9004808DD
:100AD000D0004708CF004608CE004508CD00B52419
:100AE0000008BC00840A0008BD00840A0008BE009B
:100AF000840A0008BF00FD308407F708031D932D0A
:100B0000400A43020319932D41080319952D0F390B
:100B1000430203198D2D0318C52DC11BC52D411B83
:100B2000952D2030C12D2030C105C11EA32DC1122D
:100B30004008031DC1037708C1002D30C90098206B
:100B40004108F700C10140084302031DB12D770899
:100B5000C1002E30C90098204108F7002030C1059F
:100B600000303030C11EC12DC1124008031DC10329
:100B70007708C1002D30C90098204108F700C10155
:100B80003030F7077708C90098204808CC0047089C
:100B9000CB004608CA004508C900D001CF01CE01EC
:100BA0000A30CD00B5247A08C8007908C700780853
:100BB000C6007708C500C30B5F2D08004E08D5009E
:100BC0005208D506D51FE92D03110310CE1B0314BF
:100BD0001C2E4E08D5005108D6004D08D602031928
:100BE000F72DD51F1C2E0308013A83001C2E520836
:100BF000D6004E08D6020319032ED51F1C2E03085B
:100C0000013A83001C2E5308D6004F08D602031960
:100C10000F2ED51F1C2E0308013A83001C2E5408EA
:100C2000D6005008D60203191B2ED51F1C2E030810
:100C3000013A83001C2E0310080080308318D6066A
:100C4000DB01DC015208DA005608DA065108031904
:100C50000D2FD900F70055080319162FD9020319D3
:100C6000B22E031C702E5608DF00DF175708DE0077
:100C70005808DD00DC010310DF0CDE0CDD0CDC0CA1
:100C8000D90B3A2EDA1F472E5B142A2F5B1059100E
:100C90005B165430840083133F2F5B12DA1B5A2EED
:100CA000591C652EDF0CDE0CDD0CDC0CF70A031979
:100CB000252F652EDF1B682E0310DC0DDD0DDE0DEC
:100CC000DF0DF7030319252F5A2E5B17D22E5B1366
:100CD0005208DA00DA1F6E2EDF171E2FDF131E2FC9
:100CE0005508D900F7005108D9025208DF00DF1774
:100CF0005308DE005408DD00DC010310DF0CDE0CBD
:100D0000DD0CDC0CD90B7C2EDA1F892EDB142A2F8C
:100D1000DB105910DB165830840083133F2FDB1291
:100D2000DA1B9C2E591CA72EDF0CDE0CDD0CDC0C14
:100D3000F70A0319252FA72EDF1BAA2E0310DC0D9F
:100D4000DD0DDE0DDF0DF7030319252F9C2EDB17BC
:100D5000D22EDB135608DA00DA1FB02EDF171E2F53
:100D6000DF131E2F5608DF00DF175708DE00580874
:100D7000DD00DA1FBF2EDF135B152A2F5B11DC01AC
:100D800059105430840083133F2FDA1BE82E520889
:100D9000DA00591CD22EDF0CDE0CDD0CDC0CF70A5D
:100DA0000319252FDC1FE32EDD0A031DE32EDE0AC7
:100DB000031DE32EDF0A031DE32EDF0CDE0CDD0C2A
:100DC000F70A0319252F5B1B672EDB1BA92E072FA4
:100DD0008030DF06DF1FF02E2A2F5608DA00FD2EA6
:100DE0005208DA00DF08031DFD2EDE08031DFD2E6C
:100DF000DD08031DFD2EF7011E2FDF1B072F03103B
:100E0000DC0DDD0DDE0DDF0DF70BFD2E252FDA1FBE
:100E10000B2FDF171E2FDF131E2F5508F700560864
:100E2000DF005708DE005808DD001E2F5108F700CC
:100E30005208DF005308DE005408DD005F08F800A8
:100E40005E08F9005D08FA005D2FF701F801F9016D
:100E5000FA015D2FDC01DD09DE09DF09DC09DC0AAE
:100E6000031D382FDD0A031D382FDE0A0319DF0AA0
:100E70005B18462EDB18882E5B19BE2EED2E00085F
:100E8000DD07031C492FDE0A031D492FDF0A031962
:100E9000591484030008DE07031C512FDF0A0319CD
:100EA000591484030008801F803ADF07031859147F
:100EB0005B1A4D2EDB1A8F2EC52E08003D308400A4
:100EC000831300080319712F0230F800F701F70BA4
:100ED000672FF80B662F9730F700F70B6D2F800BFD
:080EE000642F8A110A164E2E40
:101000004C10CC103F08C3003E08C2003D08C10090
:101010003C08C0003F08D0003E08CF003D08CE008D
:101020003C08CD00D401D301D201D1018A11DE25C3
:101030008A15031C1F284C144108803AC100D001B6
:10104000CF01CE017F30CD004308D4004208D30049
:101050004108D2004008D1008A11DE258A15031C00
:101060004A28D401D301D2017F30D1004308D800EF
:101070004208D7004108D6004008D5008A117623DF
:101080008A157A08C3007908C2007808C100770879
:10109000C000CC140A30D4008930D3003430D200E0
:1010A0007C30D1004308D8004208D7004108D60060
:1010B0004008D5008A1140248A157708CD007808A9
:1010C000CE007908CF007A08D000D4004F08D300B2
:1010D0004E08D2004D08D1004308D8004208D7007E
:1010E0004108D6004008D5008A1140248A157708A7
:1010F000CD007808CE007908CF007A08D0008310A0
:101100005008D4004F08D3004E08D2004D08D1003B
:101110007C30D8007930D7003530D6008130D5000A
:101120008A111D268A157A08C7007908C600780832
:10113000C5007708C4004708D4004608D300450816
:10114000D2004408D1004308D8004208D700410823
:10115000D6004008D5008A1140248A157708CD00B2
:101160007808CE007908CF007A08D000D4004F0864
:10117000D3004E08D2004D08D1004308D8004208E1
:10118000D7004108D6004008D5008A1140248A15AE
:101190007708CD007808CE007908CF007A08D00013
:1011A00083105008D4004F08D3004E08D2004D08D9
:1011B000D1003F30D8000230D7003330D600833022
:1011C000D5008A111D268A157A08C7007908C6003D
:1011D0007808C5007708C4004708D4004608D30043
:1011E0004508D2004408D1004308D8004208D7007F
:1011F0004108D6004008D5008A1140248A15770896
:10120000CD007808CE007908CF007A08D000D4004D
:101210004F08D3004E08D2004D08D1004308D80033
:101220004208D7004108D6004008D5008A11402462
:101230008A157708CD007808CE007908CF007A08A3
:10124000D00083105008D4004F08D3004E08D200BD
:101250004D08D1003330D8008C30D7001E30D60076
:101260008330D5008A111D268A157A08C7007908AF
:10127000C6007808C5007708C400D401D301D201A4
:101280007F30D1004308D8004208D7004108D6007B
:101290004008D5008A1140248A157708CD007808C7
:1012A000CE007908CF007A08D000D4004F08D300D0
:1012B0004E08D2004D08D1004308D8004208D7009C
:1012C0004108D6004008D5008A1140248A157708C5
:1012D000CD007808CE007908CF007A08D0008310BE
:1012E0005008D4004F08D3004E08D2004D08D1005A
:1012F0001B30D800E430D7003530D6008230D5001E
:101300008A111D268A157A08CB007908CA00780848
:10131000C9007708C8004B08D4004A08D300490820
:10132000D2004808D1004308D8004208D70041083D
:10133000D6004008D5008A1140248A157708CD00D0
:101340007808CE007908CF007A08D000D4004F0882
:10135000D3004E08D2004D08D1004308D8004208FF
:10136000D7004108D6004008D5008A1140248A15CC
:101370007708CD007808CE007908CF007A08D00031
:1013800083105008D4004F08D3004E08D2004D08F7
:10139000D100A430D800DB30D7006730D6008330CE
:1013A000D5008A111D268A157A08CB007908CA0053
:1013B0007808C9007708C8004B08D4004A08D30051
:1013C0004908D2004808D1004308D8004208D70095
:1013D0004108D6004008D5008A1140248A157708B4
:1013E000CD007808CE007908CF007A08D000D4006C
:1013F0004F08D3004E08D2004D08D1004308D80052
:101400004208D7004108D6004008D5008A11402480
:101410008A157708CD007808CE007908CF007A08C1
:10142000D00083105008D4004F08D3004E08D200DB
:101430004D08D1003330D8008C30D7001E30D60094
:101440008330D5008A111D268A157A08CB007908C9
:10145000CA007808C9007708C8004308D4004208C9
:10146000D3004108D2004008D1004708D800460800
:10147000D7004508D6004408D5008A1140248A15B3
:101480007708CD007808CE007908CF007A08D00020
:10149000D4004F08D3004E08D2004D08D1004B08AD
:1014A000D8004A08D7004908D6004808D5008A1154
:1014B00076238A157A08C7007908C6007808C5001F
:1014C0007708C400CC1C802A8314DB30D4000F3092
:1014D000D3004930D2007F30D1004708D8004608F9
:1014E000D7004508D6004408D5008A111D268A1564
:1014F0007A08C7007908C6007808C5007708C400D4
:101500004C1C852A4508803AC5004408F700450868
:10151000F8004608F9004708FA008A110A168C2DCF
:10200000840183131F308305713083168F000F08FE
:102010008312A01320088316870083128717831664
:1020200003170908C039890003131F129F120030DB
:10203000031788008312870188018901FF30031389
:10204000A000831603170908C039890003131F1263
:102050009F12003003178800831203131F139F136E
:1020600083169F1383121F149412A0122008831644
:102070008700831220162008831687008312A01180
:1020800020088316870001308312940000308316E5
:1020900094000108C739083881008312900100308C
:1020A000F800920000308316920083122015200859
:1020B000831687008312970183169B019C010130D0
:1020C0009D008312031787018801890104308D0068
:1020D00000308F000A120313BC280A1620162008AD
:1020E0008316870000008312A0152008831687003E
:1020F00000008312071220122008831687000000B8
:1021000083128711A01120088316870038308312AC
:10211000BC000A1204210A162A30BC000A1204214B
:102120000A160130BC000A1204210A1620122008E7
:102130008316870000008312A015200883168700ED
:102140008312871DA1280000A52800002016200862
:102150008316870000008312A201A101A401A3013C
:10216000201620088316870000008312A01520087F
:10217000831687000000831207122012200883169E
:102180008700000083128711A011200883168700A2
:1021900039308312BC000A1204210A1678083B1059
:1021A00078183B1420122008831687000000831241
:1021B000A0152008831687008312871DDD280000E4
:1021C000E128000020162008831687000000013057
:1021D0008312BB062012200883168700000083129A
:1021E000A0152008831687008312871DF52800009C
:1021F000F9280000201620088316870000008312AB
:10220000201620088316870000008312A0152008DE
:1022100083168700000083120712201220088316FD
:102220008700000083128711A01120088316870001
:1022300038308312BC000A1204210A160130BC0097
:102240000A1204210A1620162008831687000000AF
:102250008312A01520088316870000008312871DB3
:102260002F290712201220088316870000008312EE
:102270008711A01120088316870039308312BC0013
:102280000A1204210A16F7010A124E210A167808CA
:10229000B600201220088316870000008312A015C4
:1022A0002008831687008312871D542900005829AF
:1022B00000002016200883168700000083122016D5
:1022C00020088316870000008312A01520088316BB
:1022D000870000008312071220122008831687004F
:1022E000000083128711A011200883168700383060
:1022F0008312BC000A1204210A160230BC000A1222
:1023000004210A1620162008831687000000831275
:10231000A01520088316870000008312871D8E29D0
:1023200007122012200883168700000083128711ED
:10233000A01120088316870039308312BC000A12CE
:1023400004210A16F7010A124E210A167808B50070
:10235000201220088316870000008312A015200891
:10236000831687008312871DB3290000B729000058
:1023700020162008831687000000831220162008EC
:102380008316870000008312A0152008831687009B
:102390000000831207122012200883168700000015
:1023A00083128711A011200883168700383083120A
:1023B000BC000A1204210A160330BC000A120421D0
:1023C0000A16201620088316870000008312A01525
:1023D00020088316870000008312871DED2907124D
:1023E0002012200883168700000083128711A01195
:1023F00020088316870039308312BC000A1204219A
:102400000A16F7010A124E210A167808B80020129F
:1024100020088316870000008312A0152008831669
:1024200087008312871D122A0000162A000020163A
:1024300020088316870000008312201620088316C8
:10244000870000008312A015200883168700000073
:1024500083120712201220088316870000008312BF
:102460008711A01120088316870038308312BC0022
:102470000A1204210A160430BC000A1204210A16AA
:10248000201620088316870000008312A01520085C
:102490008316870000008312871D4C2A0712201222
:1024A000200883168700000083128711A0112008DE
:1024B0008316870039308312BC000A1204210A16E1
:1024C000F7010A124E210A167808B70020122008D8
:1024D0008316870000008312A0152008831687004A
:1024E0008312871D712A0000752A0000201620081B
:1024F00083168700000083122016200883168700A9
:1025000000008312A01520088316870000008312A4
:1025100007122012200883168700000083128711FB
:10252000A01120088316870038308312BC000A12DD
:1025300004210A160530BC000A1204210A162016CE
:1025400020088316870000008312A0152008831638
:10255000870000008312871DAB2A07122012200873
:1025600083168700000083128711A01120088316AC
:10257000870039308312BC000A1204210A16F701C1
:102580000A124E210A167808BA0020122008831673
:10259000870000008312A01520088316870083128D
:1025A000871DD02A0000D42A000020162008831698
:1025B0008700000083122016200883168700000081
:1025C0008312A015200883168700000083120712CB
:1025D0002012200883168700000083128711A011A3
:1025E00020088316870038308312BC000A120421A9
:1025F0000A160630BC000A1204210A16201620080A
:102600008316870000008312A01520088316870018
:1026100000008312871D0A2B071220122008831640
:102620008700000083128711A011200883168700FD
:1026300039308312BC000A1204210A16F7010A126B
:102640004E210A167808B900201220088316870048
:1026500000008312A0152008831687008312871DAF
:102660002F2B0000332B0000201620088316870034
:1026700000008312201620088316870000008312B2
:10268000A01520088316870000008312071220126D
:10269000200883168700000083128711A0112008EC
:1026A0008316870038308312BC000A1204210A16F0
:1026B000BC010A1204210A1620162008831687007E
:1026C00000008312A01520088316870000008312E3
:1026D000871D682B07122012200883168700000030
:1026E00083128711A01120088316870039308312C6
:1026F000BC000A1204210A16F7010A124E210A161A
:102700007808B90020122008831687000000831281
:10271000A0152008831687008312871D8D2B0000CB
:10272000912B00002016200883168700000010302F
:10273000831203178D0000308F000310063003133F
:10274000BD000A1293210A163508BC001B30BD00DB
:102750000A12F7210A16143003178D0000308F007B
:1027600003100D300313BD000A1293210A161B300B
:1027700003178D0000308F00031006300313BD00D7
:102780000A1293210A163608BC001B30BD000A123B
:10279000F7210A161F3003178D0000308F00031039
:1027A0000D300313BD000A1293210A1626300317B9
:1027B0008D0000308F00031006300313BD000A1295
:1027C00093210A163708BC001B30BD000A12F721FE
:1027D0000A162A3003178D0000308F0003100D30C9
:1027E0000313BD000A1293210A16313003178D001E
:1027F00000308F00031006300313BD000A1293212E
:102800000A163808BC001B30BD000A12F7210A1650
:10281000353003178D0000308F0003100D30031387
:10282000BD000A1293210A163C3003178D000030B8
:102830008F00031006300313BD000A1293210A16FD
:102840003908BC001B30BD000A12F7210A164030BF
:1028500003178D0000308F0003100D300313BD00EF
:102860000A1293210A16473003178D0000308F009B
:10287000031006300313BD000A1293210A163A080A
:10288000BC001B30BD000A12F7210A164B3003179B
:102890008D0000308F0003100D300313BD000A12AD
:1028A00093210A16BD013608BC00BD00BC013508E5
:1028B0003C07A7003D08A8000318A80ABD01380876
:1028C000BC00BD00BC0137083C07A9003D08AA00B8
:1028D0000318AA0ABD013A08BC00BD00BC013908B2
:1028E0003C07AB003D08AC000318AC0A2808BD004B
:1028F0002708BC00BF010430BE000A122C220A16B1
:102900007908A8007808A7002A08BD002908BC009B
:10291000BF010430BE000A122C220A167908AA0050
:102920007808A9002C08BD002B08BC00BF010430AA
:10293000BE000A122C220A167908AC007808AB00F7
:1029400000303B180130BC00523003178D000030BE
:102950008F00031006300313BD000A1293210A16DC
:102960003C08BD001F30BE000A126A2A0A16563003
:1029700003178D0000308F0003100D300313BD00CE
:102980000A1293210A165D3003178D0000308F0064
:10299000031007300313BD000A1293210A161030EA
:1029A00084002808BD002708BC000A12D1220A169C
:1029B000623003178D0000308F0003100C300313BA
:1029C000BD000A1293210A16693003178D000030EA
:1029D0008F00031007300313BD000A1293210A165B
:1029E000103084002A08BD002908BC000A12D12238
:1029F0000A166E3003178D0000308F0003100C3064
:102A00000313BD000A1293210A16753003178D00B7
:102A100000308F00031007300313BD000A1293210A
:102A20000A16103084002C08BD002B08BC000A12C6
:102A3000D1220A167A3003178D0000308F00031060
:102A40000C300313BD000A1293210A162A08C10094
:102A50002908C0000A1251230A167708BC0078081A
:102A6000BD007908BE007A08BF002C08C1002B0801
:102A7000C0000A1251230A163F08D4003E08D300B2
:102A80003D08D2003C08D1007A08D8007908D70068
:102A90007808D6007708D5000A1276230A167A0835
:102AA000B0007908AF007808AE007708AD0081303B
:102AB00003178D0000308F00031004300313BD0096
:102AC0000A1293210A16093084003008BF002F082B
:102AD000BE002E08BD002D08BC000230C0000A1246
:102AE000F7240A162030C9000A1298200A160D3061
:102AF000C9000A1298200A160A30C9000A12982042
:102B00000A163008BF002F08BE002E08BD002D0891
:102B1000BC000A128A1500280A168A117A08B40025
:102B20007908B3007808B2007708B100883003173D
:102B30008D0000308F00031005300313BD000A1212
:102B400093210A16093084003408BF003308BE0000
:102B50003208BD003108BC000230C0000A12F72460
:102B60000A162030C9000A1298200A160D30C90032
:102B70000A1298200A160A30C9000A1298200A166A
:102B80003408D4003308D3003208D2003108D10011
:102B9000C330D800F530D7004830D6008030D5009B
:102BA0000A1276230A167708BC007808BD00790857
:102BB000BE007A08BF00D4003E08D3003D08D20012
:102BC0003C08D100D801D7013430D6008630D5007A
:102BD0000A1240240A167A08B4007908B30078086B
:102BE000B2007708B1003108F7003208F800330866
:102BF000F9003408FA00F8133408B4003308B300BD
:102C00007808B2003108B1008314D401D301343004
:102C1000D2008530D1003408D8003308D7003208FC
:102C2000D6003108D5000A121D260A167A08B4000B
:102C30007908B3007808B2007708B1009030031724
:102C40008D0000308F00031005300313BD000A1201
:102C500093210A16093084003408BF003308BE00EF
:102C60003208BD003108BC000230C0000A12F7244F
:102C70000A162030C9000A1298200A160D30C90021
:102C80000A1298200A160A30C9000A1298200A1659
:102C90000830BC00FA30BD000A125E2F0A16BC0BC9
:062CA0004A2EAC2863007F
:04400E00F52CFF3F4F
:00000001FF
